:1000000012C0189518951895189518951895189563
:10001000AAC6D0C2189518951895189518951895D0
:100020001895189518958FE58DBFC8E3E0E24E2E20
:1000300084E08EBFD4E0F4E05F2EA89584B7082E4C
:10004000877F84BF88E1992781BD91BDEEEFF3E002
:10005000A0E6B0E088278D933197E9F76624A09851
:10006000A89AA198A99AA298AA9A8FEF81BB8FEF1C
:1000700087BB86E886B980E487B981E08093620017
:1000800000916200063010F009F015C08BE090E09E
:10009000A2E6B0E0AD90BB24A3E6B0E0AA0CBB1C86
:1000A000AA0DBB1D8D939C93A2E6B0E08C918F5F4F
:1000B0008C9308F4E5CFEAE1F0E0A2E9B0E091E04A
:1000C00098DC989957C081E08093620000916200AB
:1000D000083C10F009F04EC000916200063909F0AA
:1000E0003CC080918C00806880938C00A2E9B0E0D5
:1000F0008C9198E089278C93EAE1F0E0A2E9B0E0E6
:1001000091E07BE765DC00919200003009F00EC0C1
:1001100092989698C798C2989098C6989798C598BC
:10012000939A949A919A959AC09AC19A0091920042
:10013000083009F00EC0929A969AC79AC29A909A7D
:10014000C69A979AC59A9398949891989598C098BA
:10015000C1988CED95E072DA0DC0989B01C00AC081
:100160008AE090E06BDAA2E6B0E08C918F5F8C932E
:1001700008F4ACCFE4E1F0E0A0E1B0E037DC0F3F01
:1001800009F05AC086E490E0A5E7B0E08D939C9317
:1001900082E390E0A3E7B0E08D939C9380E590E04C
:1001A000ABE7B0E08D939C938CE390E0A9E7B0E0DF
:1001B0008D939C9388E0809392008EEE80938F00C5
:1001C0008EEE80939000E0E0F0E0A3E7B0E092E0F4
:1001D0007BE7FEDBE5E0F0E0A5E7B0E092E07BE75F
:1001E000F7DBEAE0F0E0A9E7B0E092E07BE7F0DBE4
:1001F000EEE0F0E0ABE7B0E092E07BE7E9DBE0E1E6
:10020000F0E0AFE8B0E091E07BE7E2DBE1E1F0E0D5
:10021000A0E9B0E091E07BE7DBDBEAE1F0E0A2E916
:10022000B0E091E07BE7D4DBE4E1F0E0A0E1BB27C4
:1002300084E68C937BE7C9DBE0E0F0E0A3E7B0E085
:1002400092E0D7DBE5E0F0E0A5E7B0E092E0D1DBBB
:10025000EAE0F0E0A9E7B0E092E0CBDBEEE0F0E02E
:10026000ABE7B0E092E0C5DBE0E1F0E0AFE8B0E0A2
:1002700091E0BFDBE1E1F0E0A0E9B0E091E0B9DBC3
:1002800083E083BF80E08FBD81E08EBD789489B725
:10029000816089BF89B7846089BF83E083BF81E0C3
:1002A0008EBD379A82E3809362000091620008322B
:1002B00010F009F001C03DC0882783BF8EB5887F4C
:1002C0008EBD80918C00826080938C0080E0809352
:1002D000620007B1007F056007B9BFD9A0EAB0E0AE
:1002E0008D939C9307B1007F046007B9B6D9A2EA49
:1002F000B0E08D939C93E0EAF0E0D190E0808FEF46
:10030000E7FE8827F82E082F1DDAA8E9B0E04BDABF
:10031000E2EAF0E0D190E0808FEFE7FE8827F82E48
:10032000082F10DAACE9B0E03EDA83E083BF81E069
:100330008EBDACE8B0E08C9181FB0EF090C0809156
:100340008C008D7F80938C00E8E9F0E0D7D9E0E065
:10035000FAE101DB09DB08F40DC0E0E0FAE1FBDAC9
:10036000E8E9F0E0CBD996DAEDE0F0E0A8E9B0E01A
:1003700020DB05C0A8E9B0E0E4E0FAE10FDBE8E04B
:10038000FAE1E9DAE8E9F0E0B9D92DDAEDE0F0E0F8
:10039000A8E9B0E00EDBE8E9F0E0B0D9ECE0FAE182
:1003A000DADAE2DA10F009F001C005C0A8E9B0E03D
:1003B000ECE0FAE1F3DAECE9F0E0A0D9E0E0FAE110
:1003C000CADAD2DA08F40DC0E0E0FAE1C4DAECE906
:1003D000F0E094D95FDAEDE0F0E0ACE9B0E0E9DA22
:1003E00005C0ACE9B0E0E4E0FAE1D8DAE8E0FAE12F
:1003F000B2DAECE9F0E082D9F6D9EDE0F0E0ACE970
:10040000B0E0D7DAECE9F0E079D9ECE0FAE1A3DA90
:10041000ABDA10F009F001C005C0ACE9B0E0ECE0E7
:10042000FAE1BCDA882783BF8EB5887F8EBDE8E904
:10043000F0E026D9A1E7B0E0EE0C000FE794DD92E2
:10044000EC92ECE9F0E01CD9A7E7B0E0EE0C000F6D
:10045000E794DD92EC9283E083BF81E08EBDA5E757
:10046000B0E04D915C91A3E7B0E00D911C910417B1
:10047000150708F021C0A3E7B0E04D915C91A1E71A
:10048000B0E00D911C910417150714F009F003C09A
:1004900081E080937D00A5E7B0E04D915C91A1E7FC
:1004A000B0E00D911C91041715070CF001C003C0BA
:1004B00080E080937D0020C0A3E7B0E04D915C9187
:1004C000A1E7B0E00D911C91041715070CF001C0D5
:1004D00003C081E080937D00A5E7B0E04D915C9181
:1004E000A1E7B0E00D911C910417150714F009F075
:1004F00003C080E080937D0000917D00013009F011
:1005000002C0C39A01C0C398ABE7B0E04D915C91C3
:10051000A9E7B0E00D911C910417150708F021C060
:10052000A9E7B0E04D915C91A7E7B0E00D911C9177
:100530000417150714F009F003C081E080937E00D2
:10054000ABE7B0E04D915C91A7E7B0E00D911C9155
:10055000041715070CF001C003C080E080937E00F3
:1005600020C0A9E7B0E04D915C91A7E7B0E00D9104
:100570001C91041715070CF001C003C081E08093A3
:100580007E00ABE7B0E04D915C91A7E7B0E00D9144
:100590001C910417150714F009F003C080E0809344
:1005A0007E0000917E00013009F002C0C49A01C0B3
:1005B000C4987BCE0F921F922F923F924F925F92E0
:1005C0007F92AF92BF920F931F932F933F934F93BE
:1005D0005F936F937F938F939F93AF93BF93CF93CB
:1005E000DF93EF93FF938FB78F9300918B000030D1
:1005F00081E009F480E08F93ACE8B0E08C9185FB5A
:1006000081E00EF480E09F918923882309F403C0E0
:10061000ADE8B0E0BFD7ADE8B0E00D911C91083572
:100620005BE1150710F009F001C009C080E090E01F
:10063000ADE8B0E08D939C9380E080938B00882799
:1006400083BF00918B00003009F011C0A1E7B0E03A
:100650008D919C91A5E8B0E08D939C93A7E7B0E0C5
:100660008D919C91A7E8B0E08D939C934FC0013091
:1006700009F011C0A3E7B0E08D919C91A5E8B0E02E
:100680008D939C93A7E7B0E08D919C91A7E8B0E093
:100690008D939C933BC0023009F011C0A5E7B0E0F8
:1006A0008D919C91A5E8B0E08D939C93A7E7B0E075
:1006B0008D919C91A7E8B0E08D939C9327C0033067
:1006C00009F011C0A1E7B0E08D919C91A5E8B0E0E0
:1006D0008D939C93A9E7B0E08D919C91A7E8B0E041
:1006E0008D939C9313C0043009F010C0A1E7B0E0D3
:1006F0008D919C91A5E8B0E08D939C93ABE7B0E021
:100700008D919C91A7E8B0E08D939C93ACE8B0E00C
:100710008C9183FB0EF45FC0A5E8B0E08D919C91B5
:10072000AFE7B0E08D939C93AFE7B0E08D919C91E3
:10073000A3E8B0E08D939C9383E0809363004091A5
:10074000630001E0041710F009F025C0AFE7B0E046
:100750000D911C914AE050E02ED7A3E6B0E0AD9099
:10076000BB24A3E6B0E0AA0CBB1CAA0DBB1D0D93D5
:100770001C93AFE7B0E00D911C914AE050E01BD70D
:10078000AFE7B0E04D935C9380916300815080931C
:10079000630008F0D4CFA3E8B0E00D911C910436BB
:1007A00050E015070CF401C006C08BE090E0A5E610
:1007B000B0E08D939C93A3E8B0E00D911C910A30BA
:1007C00050E015070CF401C006C08BE090E0A7E6EE
:1007D000B0E08D939C93ACE8B0E08C9182FB0EF47A
:1007E0005FC0A7E8B0E08D919C91A1E8B0E08D9347
:1007F0009C93A1E8B0E08D919C91A3E8B0E08D932B
:100800009C9386E0809363004091630004E00417AA
:1008100010F009F025C0A1E8B0E00D911C914AE06C
:1008200050E0C9D6A3E6B0E0AD90BB24A3E6B0E0AB
:10083000AA0CBB1CAA0DBB1D0D931C93A1E8B0E034
:100840000D911C914AE050E0B6D6A1E8B0E04D937E
:100850005C938091630081508093630008F0D4CF53
:10086000A3E8B0E00D911C91043650E015070CF49C
:1008700001C006C08BE090E0ABE6B0E08D939C93A6
:10088000A3E8B0E00D911C910A3050E015070CF47C
:1008900001C006C08BE090E0ADE6B0E08D939C9384
:1008A00000919200003009F007C0939894989198B5
:1008B0009598C098C19806C0939A949A919A959ADF
:1008C000C09AC19AA0E6B0E08C918F5F8C930091A2
:1008D0006000063010F009F001C003C081E0809391
:1008E000600080E08093610090D1A4E6B0E08C913C
:1008F00080FBA2E3B0E08C9182F98C9386D1A4E6D0
:10090000B0E08C9180FBA2E3B0E08C9186F98C93EF
:100910007CD1A4E6B0E08C9180FBA8E3B0E08C91A0
:1009200087F98C9372D1A4E6B0E08C9180FBA8E3A8
:10093000B0E08C9182F98C9368D1A4E6B0E08C9100
:1009400080FBA2E3B0E08C9180F98C935ED1A4E6A9
:10095000B0E08C9180FBA8E3B0E08C9186F98C9399
:1009600054D1A4E6B0E08C9180FBA2E3B0E08C917E
:1009700087F98C9300916000013009F02FC000913D
:100980009200003009F013C0919AACE8B0E08C916D
:1009900083FB0EF40AC0AFE8B0E08C9183FBA8E3C0
:1009A000B0E08C9185F98C9301C0C59A16C09198DE
:1009B000ACE8B0E08C9183FB0EF40EC0AFE8B0E081
:1009C0008C9183FBA8E3B0E08C9185F98C9388B37C
:1009D00090E2892788BB01C0C598F9C0023009F0B0
:1009E0002FC000919200003009F013C0949AACE837
:1009F000B0E08C9183FB0EF40AC0AFE8B0E08C91BC
:100A000082FBA8E3B0E08C9185F98C9301C0C59A74
:100A100016C09498ACE8B0E08C9183FB0EF40EC045
:100A2000AFE8B0E08C9182FBA8E3B0E08C9185F94F
:100A30008C9388B390E2892788BB01C0C598C7C052
:100A4000033009F02FC000919200003009F013C06C
:100A5000939AACE8B0E08C9183FB0EF40AC0AFE847
:100A6000B0E08C9181FBA8E3B0E08C9185F98C9388
:100A700001C0C59A16C09398ACE8B0E08C9183FB96
:100A80000EF40EC0AFE8B0E08C9181FBA8E3B0E0BB
:100A90008C9185F98C9388B390E2892788BB01C03B
:100AA000C59895C0043009F02FC000919200003025
:100AB00009F013C0C19AACE8B0E08C9182FB0EF44F
:100AC0000AC0A0E9B0E08C9183FBA8E3B0E08C9170
:100AD00085F98C9301C0C59A16C0C198ACE8B0E006
:100AE0008C9182FB0EF40EC0A0E9B0E08C9183FBE8
:100AF000A8E3B0E08C9185F98C9388B390E28927C4
:100B000088BB01C0C59863C0053009F02FC00091B3
:100B10009200003009F013C0C09AACE8B0E08C91AC
:100B200082FB0EF40AC0A0E9B0E08C9182FBA8E33E
:100B3000B0E08C9185F98C9301C0C59A16C0C0981D
:100B4000ACE8B0E08C9182FB0EF40EC0A0E9B0E0FE
:100B50008C9182FBA8E3B0E08C9185F98C9388B3EB
:100B600090E2892788BB01C0C59831C0063009F0E2
:100B70002EC000919200003009F013C0959AACE8A5
:100B8000B0E08C9182FB0EF40AC0A0E9B0E08C9139
:100B900081FBA8E3B0E08C9185F98C9301C0C59AE4
:100BA00016C09598ACE8B0E08C9182FB0EF40EC0B4
:100BB000A0E9B0E08C9181FBA8E3B0E08C9185F9CD
:100BC0008C9388B390E2892788BB01C0C59883E0E5
:100BD00083BF8F918FBFFF91EF91DF91CF91BF9135
:100BE000AF919F918F917F916F915F914F913F91C5
:100BF0002F911F910F91BF90AF907F905F904F907A
:100C00003F902F901F900F901895A0E6B0E0AD9008
:100C1000BB24A3E6B0E0AA0CBB1CAA0DBB1D0C9123
:100C200047E0049FA4E6B0E00C920091610040917F
:100C30006400040FA4E6B0E00C9300919200003031
:100C400009F00AC0E6E7FCE0A4E6B0E08C91992741
:100C5000A4E6B0E0ABD609C0EEEEFCE0A4E6B0E05E
:100C60008C919927A4E6B0E0A1D6A1E6B0E08C91E2
:100C70008F5F8C93089500000000000001010000C8
:100C8000010101010000010000010000000000015D
:100C9000010001000001010000000100000100004E
:100CA000000100000000000000000101010100003F
:100CB000000000000000000000010000010101012F
:100CC0000101000101010101010101010100000018
:100CD000010101000100010000010101000000000C
:100CE00001010000000001010101000100000101FB
:100CF00001010101000001010000000001010001EB
:100D000001000101010101000001000101000001D9
:100D100001010001010001010100010101010101C6
:100D200001010000000001010101010101010101B7
:100D300001000101000000000000010000000000AF
:100D4000000000000001010100000001000100019D
:100D5000010000000101010100000101010100008A
:100D60000000010001000F921F922F923F924F92BC
:100D70005F927F92AF92BF920F931F932F933F93F7
:100D80004F935F936F937F938F939F93AF93BF9393
:100D9000CF93DF93EF93FF938FB78F93A2E6B0E0EB
:100DA0008C918F5F8C938EB5887F8EBDA3E3B0E06E
:100DB0000C9100FB81E00EF480E08F93ACE8B0E092
:100DC0008C9187FB81E00EF480E09F9189238F93C3
:100DD000A3E3B0E00C9101FB81E00EF080E09F9175
:100DE00089238F93A3E3B0E00C9102FB81E00EF026
:100DF00080E09F918923882309F401C0B4D0ACE836
:100E0000B0E08C9184FB81E00EF080E08F93A3E34F
:100E1000B0E00C9100FB81E00EF080E09F9189230F
:100E2000882309F406C0999901C0DED29A9901C0BD
:100E30002CD3A3E3B0E00C9100FB81E00EF480E042
:100E40008F93A3E3B0E00C9101FB81E00EF480E00E
:100E50009F9189238F9300918B00003081E009F0EE
:100E600080E09F9189238F93ACE8B0E08C9186FB62
:100E700081E00EF480E09F918923882309F401C06A
:100E80005DD3A3E3B0E00C9100FB81E00EF480E0C1
:100E90008F93A3E3B0E00C9102FB81E00EF480E0BD
:100EA0009F9189238F9300918B00003081E009F09E
:100EB00080E09F9189238F93ACE8B0E08C9186FB12
:100EC00081E00EF480E09F918923882309F401C01A
:100ED0004BD3A3E3B0E00C9100FB81E00EF080E087
:100EE0008F93A3E3B0E00C9101FB81E00EF080E072
:100EF0009F9189238F93A3E3B0E00C9102FB81E0E3
:100F00000EF080E09F918923882309F405C0809129
:100F10008C008F7780938C00989B05C080918C000B
:100F20008F7B80938C0081E08EBD83E083BF8F91A7
:100F30008FBFFF91EF91DF91CF91BF91AF919F91C3
:100F40008F917F916F915F914F913F912F911F9161
:100F50000F91BF90AF907F905F904F903F902F90F8
:100F60001F900F901895789489B7816089BF83E0AE
:100F700083BF80918C00806180938C0080918C0075
:100F8000806880938C0080E090E0ADE8B0E08D93C5
:100F90009C93A5E7B0E04D915C91A3E7B0E00D9183
:100FA0001C910417150781E009F080E08F93ABE7EF
:100FB000B0E04D915C91A9E7B0E00D911C91041750
:100FC000150781E009F080E09F91892B882309F4BF
:100FD00001C0FDD0ABE8B0E08C918F5F8C930091A5
:100FE0008B00043010F009F001C003C080E0809352
:100FF0008B0000918B00003009F043C080918C0081
:10100000886080938C0080918C00846080938C0039
:101010008AE090E0A5E6B0E08D939C938AE090E0B2
:10102000A7E6B0E08D939C938AE090E0A9E6B0E05B
:101030008D939C938AE090E0ABE6B0E08D939C9317
:101040008AE090E0ADE6B0E08D939C938AE090E07A
:10105000AFE6B0E08D939C9380918C008F7E80935F
:101060008C0084EF91E0EAD28EB5887F8EBD882710
:1010700083BFEEE0F0E0ABE7B0E092E07BE7A8D41E
:101080009BC0013009F01BC080918C008860809368
:101090008C0081E090E0A9E6B0E08D939C938DE018
:1010A00090E0A7E6B0E08D939C9380E090E0A5E609
:1010B000B0E08D939C9384EF91E0C0D27DC002306C
:1010C00009F027C080918C00886080938C0081E0BB
:1010D00090E0A9E6B0E08D939C938EE090E0A7E6C7
:1010E000B0E08D939C9380E090E0A5E6B0E08D9316
:1010F0009C9384EF91E0A2D28EB5887F8EBD882725
:1011000083BFE0E0F0E0A3E7B0E092E07BE760D4EB
:1011100053C0033009F027C080918C008460809315
:101120008C0082E090E0AFE6B0E08D939C938DE080
:1011300090E0ADE6B0E08D939C9380E090E0ABE66C
:10114000B0E08D939C9384EF91E078D28EB5887F48
:101150008EBD882783BFE5E0F0E0A5E7B0E092E030
:101160007BE736D429C0043009F026C080918C007A
:10117000846080938C0082E090E0AFE6B0E08D93D5
:101180009C938EE090E0ADE6B0E08D939C9380E080
:1011900090E0ABE6B0E08D939C9384EF91E04ED26B
:1011A0008EB5887F8EBD882783BFEAE0F0E0A9E78F
:1011B000B0E092E07BE70CD480918C00877F809335
:1011C0008C0080918C008B7F80938C00089580919F
:1011D0008C00806280938C00A5E7B0E04D915C911B
:1011E000A3E7B0E00D911C910417150709F059C051
:1011F00080918C00886080938C008FE090E0A5E661
:10120000B0E08D939C9380E190E0A7E6B0E08D93F1
:101210009C9380E190E0A9E6B0E08D939C9384EFED
:1012200091E00CD28BE090E0A5E6B0E08D939C932A
:101230008BE090E0A7E6B0E08D939C938BE090E08C
:10124000A9E6B0E08D939C9384EF91E0F7D18FE015
:1012500090E0A5E6B0E08D939C9380E190E0A7E656
:10126000B0E08D939C9380E190E0A9E6B0E08D938F
:101270009C9384EF91E0E2D18BE090E0A5E6B0E0B2
:101280008D939C938BE090E0A7E6B0E08D939C93C8
:101290008BE090E0A9E6B0E08D939C9384EF91E021
:1012A000CDD1ABE7B0E04D915C91A9E7B0E00D91F5
:1012B0001C910417150709F059C080918C008460B7
:1012C00080938C008FE090E0ABE6B0E08D939C9330
:1012D00080E190E0ADE6B0E08D939C9380E190E0FA
:1012E000AFE6B0E08D939C9384EF91E0A7D18BE0C3
:1012F00090E0ABE6B0E08D939C938BE090E0ADE6A0
:10130000B0E08D939C938BE090E0AFE6B0E08D93DE
:101310009C9384EF91E092D18FE090E0ABE6B0E057
:101320008D939C9380E190E0ADE6B0E08D939C932B
:1013300080E190E0AFE6B0E08D939C9384EF91E084
:101340007DD18BE090E0ABE6B0E08D939C938BE099
:1013500090E0ADE6B0E08D939C938BE090E0AFE63B
:10136000B0E08D939C9384EF91E068D100918B0065
:10137000003009F001C027C0013009F007C0E0E0EB
:10138000F0E0A3E7B0E092E034D31DC0023009F0F2
:1013900007C0E5E0F0E0A5E7B0E092E02AD313C093
:1013A000033009F007C0EAE0F0E0A9E7B0E092E01E
:1013B00020D309C0043009F006C0EEE0F0E0ABE74E
:1013C000B0E092E016D380918B00815080938B0027
:1013D00080E090E0ADE8B0E08D939C9380918C002C
:1013E0008F7D80938C000895789489B7816089BF40
:1013F00083E083BF80E090E0ADE8B0E08D939C9304
:1014000000918B00013009F00DC0A3E7B0E00D9111
:101410001C91043650E0150708F003C0A3E7B0E0C4
:10142000B9D02FC0023009F00DC0A5E7B0E00D9192
:101430001C91043650E0150708F003C0A5E7B0E0A2
:10144000A9D01FC0033009F00DC0A9E7B0E00D918D
:101450001C91043650E0150708F003C0A9E7B0E07E
:1014600099D00FC0043009F00CC0ABE7B0E00D918B
:101470001C91043650E0150708F003C0ABE7B0E05C
:1014800089D086E490E0DAD00895789489B78160B5
:1014900089BF83E083BF80E090E0ADE8B0E08D934A
:1014A0009C9300918B00013009F00FC0A3E7B0E0DE
:1014B0000D911C91003050E0150710F009F001C0AB
:1014C00003C0A3E7B0E06DD035C0023009F00FC013
:1014D000A5E7B0E00D911C91003050E0150710F029
:1014E00009F001C003C0A5E7B0E05BD023C0033022
:1014F00009F00FC0A9E7B0E00D911C91003050E059
:10150000150710F009F001C003C0A9E7B0E049D009
:1015100011C0043009F00EC0ABE7B0E00D911C9192
:10152000003050E0150710F009F001C003C0ABE730
:10153000B0E037D086E490E081D0089580918C00AF
:10154000806480938C0091E0AFE8B0E08FD08EB5DE
:10155000887F8EBD882783BFE0E1F0E0AFE8B0E090
:1015600091E07BE735D2089580918C008064809370
:101570008C0091E0A0E9B0E079D08EB5887F8EBD77
:10158000882783BFE1E1F0E0A0E9B0E091E07BE7EC
:101590001FD20895ED91FC91EF5FFF4FFC93EE9306
:1015A0000895ED91FC91E150F040FC93EE93089585
:1015B00000FC10D0089503D01ED001F8F9CF00240C
:1015C000E89457FF02C009D0689400F80BD010F8D7
:1015D0000124089502D009D00895509540954F5F99
:1015E0005F4F0895E89417FF0895009510950F5FD9
:1015F0001F4F68940895352F242FE894452B11F43C
:1016000068940895512F402F0027112780E1440F3F
:10161000551F001F111F021B130B416018F4020F0E
:10162000131F4E7F8A9599F708953197F1F7089522
:10163000689462F80895E89462F80895EF93FF9330
:10164000EE27E82BE92B31F0E0EDF7E03197F1F7E9
:101650000197D1F7FF91EF910895369A3699FECF11
:10166000369A3699FECF84B195B10895903039F00D
:101670008C91880F08F481609A95D9F78C9308951E
:101680003DD0992711278F2D880F80E8F82A802FC9
:10169000881F08F41FEF41F08F57082F07FD04C083
:1016A000003240F08FEF01C08827982FD82EE82E07
:1016B000F82E09C08FE1801B082FF694E794D79489
:1016C00097950A95D1F7112351F09095D094E09415
:1016D000F09481E0980F8827D81EE81EF81E0F2D81
:1016E000FE2CED2CD92E0895D094E094F09491E046
:1016F000D90E9927E91EF91E10950895D190E19011
:10170000F190019108952191319141915191089564
:10171000102F90E8FF0C001F0927990FF7941078FD
:10172000652F90E8440F551F5927990F479560780A
:1017300000380895FF0C90E89027110F9795F794C3
:10174000092F0895102FBD2CDE2CEF2CF02E112325
:101750004AF4B094D094E094F0949FEFB91AD90A67
:10176000E90AF90A0EE1FF2039F4FE2CED2CDB2CFE
:10177000BB240850C2F76BC032F00A95BB0CDD1CCD
:10178000EE1CFF1CF9CF01D0D5CFB7FE089590E82D
:10179000B91611F4D0FE08959FEFD91AE90AF90A93
:1017A00009F403950895DD92ED92FD920C9308954E
:1017B000502F2D2D3E2D4F2D612F08952DEC3CECFB
:1017C0004CEC5DE366270FC099DFF2DFDD24EE24E9
:1017D00090E8F92E0FE307C096DF05C022273327D4
:1017E00040E251E46627552351F1002381F190DF57
:1017F00071F11627005850580894050B18F407FD8E
:1018000003C025C007FD23C0469537952795F6945C
:10181000E794D79422D0FF202AF0DD0CEE1CFF1CA9
:10182000015073F09D2D969548F0DD203AF4EE209E
:101830002AF491E0D90E9927E91EF91E7BCF07C043
:101840009FE7092FF92A9FEFD92EE92E0895DD246D
:10185000EE24FF240027112708959F929924AA249B
:10186000BB2488E1D216E306F40628F0D21AE30A74
:10187000F40A089401C08894991CAA1CBB1CDD0CB6
:10188000EE1CFF1C8A9571F7D92CEA2CFB2C9F903B
:10189000089539DF3DDF503829F090E869270CC002
:1018A0000AF045D047CF5FE322273327442701C002
:1018B0002ADF2EDF5038B1F3003899F3902F951BB3
:1018C0008BF312F434D0FACF983118F02227332753
:1018D0004427983028F0232F342F44279850F9CFED
:1018E000992329F04695379527959A95D9F7912F01
:1018F000962742F014D0B0F6F794E794D7940F5F90
:101900008BF69ECF10D051F008F4EEDEFF2052F29D
:10191000DD0CEE1CFF1C0150CBF792CF98CFD20EFE
:10192000E31EF41E0895D21AE30AF40A0895DF9222
:10193000EF92FF920F931F93D22EE32EF42E052FDA
:10194000162F6F915F914F913F912F910895C895F8
:10195000319600200895FBDF202DF9DF302DF7DFD1
:10196000402DF5DF502D089507FB00680EF40F772A
:1019700057FB50680EF45F7707FD02C057FF05C0A4
:10198000D216E306F406050708952D153E054F050A
:101990005007089591E005C092E003C094E001C0B3
:1019A00098E0D5DF0D929A95E1F70895E80FF91FB9
:1019B000F1CF94E081918D939A95E1F70895E199A3
:1019C000FECFEEBBFFBB3196089591E001C092E0DF
:1019D0007B3751F47FB7F894F2DF8D918DBBE29A9B
:1019E000E19A9A95C9F77FBF7727089591E001C0E2
:1019F00092E0E5DFE09A8DB38D939A95D1F7089543
:101A00000000244200000000333313410000C842AC
:00000001FF
